:1000000000308A00E12800002E3084000008031927
:1000100016280630A100A001A00B0C28A10B0B286C
:100020007B30A000A00B1228800B0928003485101B
:1000300005110830A000A00B1B2885120830A00075
:10004000A00B202885160830A000A00B2528003022
:1000500083168600831200340830A000A00B2E28DF
:1000600005100330A000A00B3328051485110330C0
:10007000A000A00B392885150034FF3083168600B8
:100080000000000000000000000083128514000042
:10009000000000000000000005150034FF30AA0039
:1000A000AB01AC011720A801A701A601A501A80872
:1000B000031D7928A708031D79282608753C031C11
:1000C0007928031D672825082F3C031C79282A0856
:1000D00086002C202B0886002C202C0886002C2043
:1000E0000130A5070318A60A0319A70A0319A80ACD
:1000F00057283D200C30AD00FA30AE000420AD0B87
:100100007C28AA01FF30AB00AC011720A801A70191
:10011000A601A501A808031DAC28A708031DAC284B
:100120002608753C031CAC28031D9A2825082F3C83
:10013000031CAC282A0886002C202B0886002C20C3
:100140002C0886002C200130A5070318A60A0319E5
:10015000A70A0319A80A8A283D200C30AD00FA30FE
:10016000AE000420AD0BAF28AA01AB01FF30AC00FC
:100170001720A801A701A601A501A808031DDF28D3
:10018000A708031DDF282608753C031CDF28031D74
:10019000CD2825082F3C031CDF282A0886002C20A8
:1001A0002B0886002C202C0886002C200130A50767
:1001B0000318A60A0319A70A0319A80ABD283D2097
:1001C000003484011F30830583161F149F141F15EC
:1001D0009F112030990026309800903083129800AB
:1001E000831681173F308312850000308316850007
:1001F000FF30860083128701BE30831687008C1281
:1002000083120B138B138B1B02296430AE00042066
:1002100007144E208C1E0A291A08A9002908003A42
:1002200003191629013A031918294A294E204A2987
:100230001720A801A701A601A501A808031D4829A8
:10024000A708031D48292608753C031C4829031DDF
:100250002D2925082F3C031C48298C1E2D291A08FE
:10026000A90086002C208C1E33291A08A9008600BC
:100270002C208C1E39291A08A90086002C20013058
:10028000A5070318A60A0319A70A0319A80A1D2916
:080290003D204A290A29630000
:02400E003A3F37
:00000001FF
